:02000000772E59
:08000800F000030EF10083017A
:100010000B1D1628F31B1228031085190314F40C6A
:10002000F50CF30381030B110B1C31288616061601
:10003000A20AA31A851A1F28A201A41FA403270835
:10004000220603198612220D7039A100210E8A01A1
:1000500038202505031D06120508A3000B100B19F7
:100060000A2872088A00710E8300F00E700E0900D3
:10007000820701340234043408341034203440340C
:100080008034B0000030F2008A0030088207FF346C
:100090000334FF34AF2C9F2C8A2C972C1434FF345C
:1000A0000434B52CFF34A92C2C345134FF34FF34E4
:1000B000382B082BFF34192BCB2B1F34FF34FF3484
:1000C000FF34012B3E343F342E344034422BFF3476
:1000D000123416343A342A3418341A34482BFF3484
:1000E0002134103438342D3428341D342734FF346F
:1000F0002334153439343D34FE2A4134FF34FF347F
:10010000FF34253401340B3444344534FF34FF3498
:10011000423405340D34083447344634FF34FF3458
:100120004334D72B00344C340A344834FF34FF3482
:10013000FF344F34FF344A344934FF34FF343C3405
:10014000042BE02B4B34FF344D34FF34FF34FF34A9
:100150005034FF34FF34FF34FF343434FF34FF3481
:100160008134FF3484348734FF34FF34FF348034E7
:100170008A3482348534863488341C34522B1334C8
:100180008B3483348C348D348934C12CFF34323435
:1001900020341E34FF34FF3435341C34FF34FF3434
:1001A00006341A340E3407343034FF34FF34051A61
:1001B000D72883160139031D85150319851183126C
:1001C000051EE028080064008B13F5000830F300DA
:1001D000F60129213230FF3E031DEB2883168511DD
:1001E0008312F228F3280000F528F6280000831671
:1001F000051683127508F606D720F50CF30BFA28BE
:100200007609D7200130D720051A0429E02083166B
:100210008515051683120A30F300FF308100A830DF
:100220008B006400F31F1129F50DF40D7408F7001D
:10023000F50D740DF400AB002921F6010830F8002B
:100240007408F706F40DF80B20292B08F71B08009B
:10025000922E83160512831208000130F2008A00E4
:10026000480882077B348D349F34C3000408D100D2
:100270004B21430880005108840043088313080081
:10028000C4000408D1004B210008C30051088400B9
:1002900043088313080083134408053C03185929B5
:1002A0004408553C03185D294408CA3E831784005E
:1002B000080044086A3E8400080044089A3E84000E
:1002C00008000030B200320883169B001C141A0884
:1002D0008312B10008006321B20A0800D0006F2623
:1002E0000030B40061215006CD0083169A000B083F
:1002F000B500831234088B1383169B0055309D0084
:10030000AA309D009C14B51B8B179C18852983125D
:10031000FF347521B40A0800FF3A0319FF342D1881
:10032000FF34AD1CFF342808C039031DFF342E1CD8
:10033000FF3428081C3A0319D82928082C1AA529A3
:10034000AC19B8293F18FF344F2ABF1CB229BF018E
:100350003E06031DB5293F18FF3428083D22031926
:10036000FF34822ABF14BE00FF34FF30BE00FF34CA
:100370004F1AFF343F1DD429BF013E06031DB52986
:100380003F18FF3428080C22031D812A2822031954
:10039000D7293F143D08023EC100B4002808B80028
:1003A00083224B156926FF343F15BE00FF34822A95
:1003B0003F1CFF34410834020319E729C100FF3014
:1003C00075213D08B40038088921410889213F1072
:1003D0004B116926832A8322E7292808343A031916
:1003E000F82934087F3C031C822A2808892100341C
:1003F00034084102031CFD29822AB4030034D201CF
:100400002822031908003D087F3CFF3ED200080067
:100410000630B30040160800BA000630B3004012A0
:100420003308B200BD007F3C0315031CFF346B2171
:10043000BB00FF3A0319FF346B21BC003207B30045
:10044000401A262A3B083A06031D102A0311FF34DE
:100450000630B2003208BD007F3C0315031CFF3498
:100460006B21FF3A0319372A6B21B2072A2A3D086C
:100470007C3C0311031C0315FF340C220319FF34C9
:100480003D08B4003308B20032087F3C031C4B2AFD
:100490006B218921442AFF3089210311FF340C226A
:1004A0000319FF346B218E22BC0B522AA92AFA3081
:1004B000F630CC00080028080C3A03196B2A2808EB
:1004C000343A03196F2A4408773C031C08002808B3
:1004D0003521C40A08004408C500C40108004408C6
:1004E000031DC4030800C200572242082627C20A7F
:1004F000B600420826278E22C20AB603031D792AB7
:10050000FF34832283222808A9009E308E222908E6
:10051000A8002030C7226030C722AC2AA8002808D3
:100520000C3A031D972AC522AC224830C72A280856
:10053000FF3A031D9F2AAC22A514C622AC2AAC2286
:1005400028084706031D4C080E3EC722C522AC2AC8
:10055000FF34A601A501AC01FF30A7000800AC1FC5
:100560002E15AE1608006400A612A613A81BA61727
:10057000281BA616FF30BE002808C7003F393F3AA7
:10058000A7002608A5000800A800B3220330A40095
:10059000A41FC82AFF34AC1A3734B730B02AAC1FB6
:1005A000D32A2D1BAF2CAC1A3434B430B02A4330CC
:1005B000AC1E5330B02A4430AC1E5430B02A8E30BA
:1005C000E22A8F302E18FF34A8000A30B6008F229E
:1005D000B60BE72AA92A0F30F22A0E30F22A06308B
:1005E000F22A0730AE16AD1AFC2ACD1F08002C1BCC
:1005F0000800AC1F8038B02A8030C82CCD1D2B34A9
:100600001734CD1D17342B342C112E1C2C150D2B0B
:10061000AE18D32BAC112E1CAC152C13AC1D2C1901
:100620002C17A6122C1BA616292B2C102E1C2C14B2
:10063000222BAE18152B2E1E1F2BAD15FF34AC1020
:100640002E1CAC14AC13AC1C2C18AC17A613AC1B92
:10065000A617AC12AC1F2C1BAC162C12AC1FFF340F
:100660002C1FFF342C16FF342D122E1C2D163D2B63
:10067000AE18342BAD122E1CAD162D13AD1E2D1A37
:100680002D17FF34AE1CFF34AD102E1CAD144D2BB6
:10069000AE1CFF342D102E1C2D142D11AD1C2D1849
:1006A0002D15FF34AD1D592BAD11A6102E1CA6140F
:1006B000FF343F1C2E1CFF34AD1AAC1C642B0230DF
:1006C000B400490875214F161030CF060030401B8A
:1006D00001384F1A0230682E0330F2008A003008C9
:1006E00082071E3475341E345E34FF341B344734A5
:1006F0001B345B34FF342034363420340234FF346E
:100700002234373422344234FF3433345B343334CC
:100710002634603435340734353470346034303442
:1007200070343034723462343234723432340F34D0
:1007300062340E344E344634663446340F34063454
:1007400073347334FF346034603481348A34FF345A
:1007500062346234063407344F340234423488340D
:100760008034FF3446344F345A347334FF342634E3
:1007700066340E344E34FF3473345E348534823440
:10078000FF34FF34FF34363437344F3473344F344E
:1007900047344634FF34AE18FF34AE16CD192D1E43
:1007A0002F342E157534FF34AC1EFF343634AE1C96
:1007B0004E344F1E26342E1CFF342030CA00512CDC
:1007C0004F1EE92BAE1C0C342E1CFF340230CA0025
:1007D000512CAE180C34AC18AD1EF92B2E1CFF3466
:1007E000401FF52B40134B10692E082640174B1461
:1007F000692E401F0C342E1CFF34DA250C300319EF
:100800008E2A0C308E2253267E25AC2AFF3A0319FD
:10081000FF340430F2008A002808B7001F39AF0007
:10082000B70E370C073982071C2C1C2C222C3C2CB1
:100830003D2C3C2C3C2C1C2C2808080003102F0DB0
:10084000B00008001E24B00D2F08B007CD19302CC1
:100850002D1BFF34AC1F2C1F2E2CB00A6C23AF2A8B
:100860000230B0072D1A382CAC1F2C1F2E2C2D2C2B
:10087000B00AAC1AFF342D2CFF341E242F07B00011
:10088000AE184D2DB00A4F1E4D2DB00A2E1CFF3450
:100890004D25CA00FF3A0319FF340A302F02031C0A
:1008A000732C4808023A0319662C4808003A031DC5
:1008B0005E2C4A080339031DFF34662C4808013AB0
:1008C000031D892C4A080739031DFF344A081F39C4
:1008D0000319FF344B1149084A0503194B154A08FF
:1008E000C906CC246F2E4808023A0319FF34480881
:1008F000013A031D7D2CF830842C4808003A031D72
:10090000892C4A19FF34FC30C9054A08C904CC2493
:100910006F2EFF342D1F11342E1CFF34AD1E072DFA
:100920002C3073221D25232529253425072D2D1B29
:10093000F52C2E1C9D2C0614FF340610FF34AD1A26
:10094000A72C2E1CA52C8614FF348610FF340830EB
:10095000C82C2E1CAD2C0615FF340611FF342E1C9E
:10096000B32C8615FF348611FF342E1CFF3457221A
:10097000C401450844020318A92A41218E22C40A51
:10098000B92CAD1AC72C9F304D1DFF34B02A04304E
:100990002E18AC1CFF346E29CA0149080739CA0059
:1009A0004A13491A4A17CA13C91ACA17C91D861306
:1009B000C919861783160508831238394A04831625
:1009C00085008312FF34831605100830F900851066
:1009D000031885140511EC2CED2C0515F90BE72CEB
:1009E000050807388500830108002E1CFF342D1AE6
:1009F000342DAD1AAC1CFF34C80A0330480203186A
:100A0000C8016F260130B40048087521302D6030D0
:100A10007322082210220319162D3B088E220E3055
:100A20008E223C087C2521308E220A2D64307322D0
:100A3000FF2152087C25FF308E2A693073222A302C
:100A4000CD193D308E2A6D3073221F304D1D32304E
:100A50008E2A723073223230CD1B1F308E229B2A99
:100A6000773073222D21732A773073222D21732240
:100A7000A83073220330B6004908CA000E308E2217
:100A8000CA0DB60B3E2D0530B600CA0D3230031824
:100A90001F308E22B60B452D9B2A0530F2008A00AE
:100AA00030088207CB2A3234FF34DB2A1F3400346B
:100AB000EB2A1E340134E12A1A340234EF2A1834A6
:100AC0000334FF341D340434F12A1B340534D72A8F
:100AD00033340634ED2A35340734DF2A3034FF341A
:100AE000CF2A22340134FF3406340434FF340E3468
:100AF0000834D42B07341034D900DA019325C015FB
:100B00000430B600543084000008031DC0118D2548
:100B1000840AB60B842D5808C011C0190800C325DB
:100B20008E225B22FF341030DB002730DC00AE2544
:100B3000D400E830DB000330DC00AE25D5006430A3
:100B4000DB000030DC00AE25D6000A30DB000030D0
:100B5000DC00AE25D7005908D8000800E10159088B
:100B6000DD005A08DE005B30E7266108031C080040
:100B7000E10A59301026B32DD000C325D500500E00
:100B8000C325D40008000F39D3000530F2008A00D5
:100B90005308820732341F341E341A3418341D347B
:100BA0001B343334353430343F34153412343A3452
:100BB0002A3438341726031908002B26C4011E27AF
:100BC0000319062E683010266630E7266808E6000E
:100BD0006908E700031C062E1E270319062E643041
:100BE00010266230E7261E27031D022E6208DD0054
:100BF0006308DE006830F5260318082E59301026E9
:100C0000031108006408E2006508E300031508000A
:100C1000FF30E200E300E600E7000315080066305D
:100C200084005D088000840A5E08800008006B2252
:100C3000450844020318292E4121E0002C3A0319EB
:100C4000272E6008213A0319272E03110800C40A31
:100C5000182E03150800C016122745084402031871
:100C6000080041214326C01E08005B3010260227E1
:100C70000319122F6108DB00DC015B30F526031835
:100C8000122FC40A2D2EE000E1016108C325600681
:100C90000319512EE10A6108093C0318452EC012C0
:100CA0000800C0160800C401B60145084402031834
:100CB0005F2E4121423A0319B60AC40A552EC401D7
:100CC00036080319FF340330C722B60B632EFF34F6
:100CD000CB00ED30E3204B080739E320FF3401302F
:100CE000CB0669260630C7220130CB06692E640088
:100CF0008B0183018C0107309F0085018316E8304A
:100D0000850040308600FF3081001C158C01831265
:100D1000FF30AA00860002306221C900CC240130D5
:100D20006221C800A922A201AD01AC01C101C40128
:100D3000C501C001BF01CF01FF30BE00F2018A0131
:100D4000CB01FF30E3200721072157226121CD008D
:100D5000AE0183010721E03A0319AE142B08F03AE3
:100D600003192E142B08E13A03192E1690302B028A
:100D70000318A92E2B084120A800AE1E0624A800A7
:100D80002D198C21A800FF3A0319DE2E2E19CE2E24
:100D90003F30A8052C08C039A804E226C8222E1C22
:100DA000D32EAC22A62E3F1CD92EED21FF3A0319DB
:100DB000A62E5B22B3220330A400A62EC82226084A
:100DC000A500A62E2D1E08008030A804080084006F
:100DD0000008DD020318F12E0130DE020318F12EA7
:100DE0000800840A0008DE02080084000008DD070D
:100DF000031CFE2E0130DE0703180800840A0008D9
:100E0000DE0708005B08DD005C08DE001527031D17
:100E1000122F5B30F5260318122F5B30F5260311D5
:100E2000031C0800DD01DE0108000310DF011927A3
:100E30001927DD0DDE0DDF0D5F0808005E30840030
:100E40000008031D0800840300080800B0000730F4
:100E5000F2008A003008820033343A343F342834B8
:100E600005343F3405340D34213438340834283403
:100E700021340A340D3412341F341B3438341B34FB
:100E80001E343534213410342A34283421341E34AD
:100E90002234323421343F341A34FF341F341F34A7
:100EA00022341E34323432343534213415342B3468
:100EB00021343A343F34283405343A340534FF348D
:100EC00003340534253442340434FF3438341534C3
:100ED00042340334053415344234043421343E346E
:100EE000003442340434213405343F344234033472
:100EF0000A34253442340734183408343E34063476
:100F00001A341534FF340934183406341F340834C5
:100F10003E3406341E341534FF3407343534083477
:100F20003E3406341E341534FF3409343534063467
:100F30001F3408343E3406341F341534FF34033470
:100F40001D341534FF3404341F3432341534FF3467
:080F500003340A341534423465
:02400E00123F5F
:084200000000000000000000B6
:04420C002F0013006C
:104210000A00080005002A0035001E0020003200B8
:1042200042000A00080005002A0033001F00320087
:10423000200032000C002E0014000A0008000500C7
:104240002A0033001A00320020001E0042000A003B
:10425000080005002A0033001E0030002000350051
:044260000C00FF004F
:00000001FF
